:020000020000FC
:020000001CC022
:02002C0073C09F
:1000380064C00FEF0DBF08E00EBF01E004B92898B7
:10004800442700E007B90FEF08B9A1D106B1009520
:100058000F73083110F4602F01C062E111272227C5
:100068007AE136E097E08AEE0DE30093890009E033
:100078000093880000E0009380000BE0009381006B
:100088000BE307BD02E004BD01E005BD02E00093FB
:100098006F0078947FD02EC0103071F5022F003099
:1000A800D9F00F50C9F0D8F7022F0130B9F000315C
:1000B800A9F0003299F0033099F0023189F0013249
:1000C80079F0073079F0093079F00E3079F0022FA5
:1000D800055071F0E8F710C05DD00CC041D10AC0DE
:1000E80042D108C044D106C046D104C048D102C09C
:1000F8004AD100C01030F1F3CFCF442329F005B125
:1001080051E0052705B918952898189513951C33BB
:10011800E9F4112723952C33C9F422276395683114
:10012800A9F466277395323091F4482F592F24D0BB
:1001380050F4482F592F26D018F4082F037019F0BF
:100148007D3121F412C07E3109F40FC014C034305F
:1001580039F0363029F0393019F03B3009F003C056
:100168007F3149F402C0703231F471E033953D308B
:1001780011F431E0019618954059514049F0E0F7E3
:10018800089408954456504019F0E0F708940895EB
:100198008894089583D05BD0682E792E48EE53E07A
:1001A8001ED0082D88D044E650E019D0082D83D001
:1001B8004AE050E014D0082D7ED0062D7CD047D0E0
:1001C8005FD045D0032F15D042D048D040D0072F5C
:1001D80010D03DD04BD03BD0062F0BD008958824AB
:1001E80099246416750620F0641A750A8394F9CF69
:1001F80008957F938F93702F88270027743618F0FF
:1002080074560395FBCF002311F081E054D00027EA
:100218007A3018F07A500395FBCF002311F4882325
:1002280011F081E048D0072F46D08F917F91089533
:1002380041E0ADD040E0ABD0089541E0A8D0A7D0D0
:10024800A6D040E0A4D00895A2D0A1D008959FD010
:100258009ED09DD09CD09BD09AD00895EEDFE8DF49
:10026800E7DFF2DF0895E4DFEFDF0895E1DFE0DFA5
:10027800DFDFDEDFE9DF0895DBDFDADFE5DF0895C2
:10028800DCDFDBDFE1DF0895D8DFD7DFD6DFDCDFB7
:100298000895CEDFCDDFCCDFD7DF0895CEDFC8DF0E
:1002A800CCDFCBDFD1DF0895C3DFC2DFC1DFC0DF22
:1002B800BFDFCADF08950130B9F00230E1F0033042
:1002C80009F1043031F1053059F1063059F10730A0
:1002D80081F10830A9F10930D1F1AFDFAEDFADDF30
:1002E800ACDFABDFB1DF0895A3DFA7DFA6DFA5DFB3
:1002F800A4DFAADF08959CDF9BDF9FDF9EDF9DDFE1
:10030800A3DF089595DF94DF93DF97DF96DF9CDF07
:1003180008958EDF8DDF8CDF8BDF8FDF95DF08950B
:100328001DD008958ADF84DF83DF82DF81DF8CDFE1
:10033800089583DF82DF7CDF7BDF7ADF85DF089546
:100348007CDF7BDF7ADF74DF73DF7EDF089575DFA4
:1003580074DF73DF72DF6CDF77DF0895A5DF089540
:100368008FDF92DF08958CDF8FDF7DDF089588DFD0
:100378008BDF82DF089584DF87DF8BDF089580DFDE
:1003880083DF74DF08957CDF7FDF8EDF089502E06E
:10039800202E04E0302E0AEB402E4A94F1F73A94CE
:0803A800E1F72A94D1F7089552
:00000001FF
